:100000000AC02BC01895189518951895189518952D
:100010001895189518958FED8DBFC0ECE0EC4E2E1D
:10002000DD275D2EEEE7F0E0A0E6B0E088278D93B7
:100030003197E9F766248FEF87BB8BE981BB84E6B4
:1000400082BB78948BB780648BBF80E088BBC79AF3
:1000500085B7806385BF8895F8CF8BB78F7B8BBFC3
:10006000E0E6F4E003D281E080936000009160005C
:100070000C3010F009F00EC0FCD1A0E6AD90ABE65C
:10008000AA0D5ED20C92F2D1A0E68C918F5F8C9378
:1000900008F4ECCF80E08093790080E080936A00E0
:1000A00080E08093690000E010E020E030E0A1E60D
:1000B0000D931D932D933C9380E0809365008D9864
:1000C000AAE79C9197FF04C0859B0EC09F779C93E5
:1000D00085990AC088E29F93992723D29F91859999
:1000E00003C090689C9397D180E488BBE1E0F0E086
:1000F000C3D1A9E78C918F5F8C9381E080936000DE
:10010000009160000C3010F009F050C000916000C8
:10011000053009F002C044C013C0063009F002C027
:100120003FC00EC0073009F002C03AC009C0083015
:1001300009F002C035C004C0093009F001C030C068
:1001400084E690E0EED180E0809378000091780022
:10015000043610F009F024C0A0E6AD90ABE6AA0D7D
:100160008C9188BB8AE090E0DCD18A98AAE79C91C8
:1001700096FF04C0829B0EC09F7B9C9382990AC00D
:1001800088E29F939927CDD19F91829903C0906473
:100190009C9318D0A8E78C918F5F8C9308F4D6CFEE
:1001A000A0E68C918F5F8C9308F4AACF0091790020
:1001B000003010F009F001C082CF8BB780648BBF94
:1001C0001895089580E080937900939AC79A84E601
:1001D00090E0A7D19398C79882E390E0A2D100273E
:1001E000A0E38C9182FB0EF401E040E0041709F0DB
:1001F00001C0F5CF00916900013009F001C02EC0A7
:1002000000916900023009F001C053C00091600004
:100210000B3009F00DC08CE588BBE2E0F0E02CD19A
:10022000A9E68C918F5F8C9380E0809365000895A0
:10023000009160000C3009F010C0E5E0F0E0A4E1AE
:1002400094E0A5D1A1E60D911D912D913C9181D114
:1002500009F002C096C001C067C03AC000916000BA
:100260000C3009F025C0E5E0F0E0A4E194E08FD186
:10027000A1E60D911D912D913C916BD109F401C026
:1002800053C074D084E588BBE2E0F0E0F5D000E034
:1002900010E020E030E0A1E60D931D932D933C93F8
:1002A00080E080936500A9E68C918F5F8C93089520
:1002B0000FC0009160000C3009F00AC0E5E0F0E0EA
:1002C000A1E694E07BE752D151D080E088BB08954D
:1002D000A5E68C918F5F8C9300916500083010F03B
:1002E00009F001C001C020C0A1E60D911D912D9122
:1002F0003C914AE050E060E070E0C4D0A1E60D938C
:100300001D932D933D93A1E60D911D912D913C914F
:10031000A0E64C9155276627772716D1A1E60D93C5
:100320001D932D933D93089581E788BBE1E0F0E0B4
:10033000A3D0ABE68C918F5F8C9389E080936700AC
:100340008FE58093680049D000916B00023010F077
:1003500009F001C007C0ECE3F0E08ED080E08093AC
:100360006B0004D083E080937900089584E690E0E8
:10037000D8D082E08093670088EC809368002DD00D
:10038000089580E080936B00F1DF80E488BB8CE20D
:1003900091E0C7D00027A0E38C9186FB0EF401E02A
:1003A00040E0041709F00BC082B390E1892782BBBB
:1003B000E1E0F0E061D083E0809379000895949AC1
:1003C000E2E0F0E059D0949880E088BBE1E0F0E012
:1003D00053D083E080937900089581E08093660094
:1003E0004091670000916600041710F009F012C0F8
:1003F000939AC79AA8E68C91992793D09398C79817
:10040000A8E68C9199278DD0A6E68C918F5F8C936E
:1004100008F4E6CF0895E3E0F0E02ED00027A0E353
:100420008C9185FB0EF401E041E0041709F001C056
:1004300013C080E788BBE5E0F0E002ED14E020E0C7
:1004400030E0A0E1BB2794E07BE790D0E1E0F0E072
:1004500013D086E488BB8ADF83E080937900089517
:10046000065B4F666D7C077F673F58798E2E9F2E07
:100470000895E82DF92D089588EE93E052D0319734
:10048000D9F7089522D006D000FC01D0089528D0D5
:1004900030D00895842F952FA62FB72F44275527A6
:1004A00066277727F1E2889409C020F4480F591F86
:1004B0006A1F7B1F769567955795479537952795C2
:1004C00017950795FA9589F708950024E89477FF22
:1004D00002C006D0689400F809D010F801240895ED
:1004E00012D04F5F5F4F6F4F7F4F0895E89437FFF3
:1004F000089500951095209530950F5F1F4F2F4F51
:100500003F4F689408954095509560957095089573
:100510003197F1F70895689462F80895E89462F8C5
:100520000895EF93FF93EE27E82BE92B31F0E8EEE7
:10053000F3E03197F1F70197D1F7FF91EF9108952B
:10054000C895319600200895040F151F261F371FE8
:10055000089504171507260737070895E199FECF78
:10056000EEBB3196089591E001C092E07B3751F4E3
:100570007FB7F894F3DF8D918DBBE29AE19A9A955B
:10058000C9F77FBF7727089591E001C092E0E6DFC9
:0C059000E09A8DB38D939A95D1F70895F1
:00000001FF
